S123E000CE100A1F0001037EB6008693B710398600B710248600B71035CEB600DF98CEB731
S123E020FFDF9ACE0000DFAC8E005FBDE357CE0041DF69B610208A03B7102086D09768CC55
S123E0403F0DDD6BBDE1B87F00A47C00A47F00A6B6103C842027358603B79800B6980084BE
S123E0607F26128612B79800B6980084022706860197A62017B6D00C810F261086AAB7D0F3
S123E0800CB6D00C81AA2604860297A67F00A5BDE34FBDE0B796A6270597A5BDE0B77F00E6
S123E0A0A5BDE39E810D271996A627F297A5BDE39E810D270C20E7BDE378CEE640BDE5184E
S123E0C0397F00A796A581012704860397A70F8E005F7F00A47C00A4BDE508863EBDE3CA17
S123E0E05FBDE544CE006B3A811827E2817F27DE810826055A2DD720E8810D26075D27174D
S123E100A7002013A7005CC1232F08CEE68ABDE51820BB812F26CA7F00C07F00967F009726
S123E1205FCE006BDFAEBDE306BDE2F1CE008E3ABDE1ADA700810D2736BDE3162731BDE260
S123E140F85CC1082F09CEE68ABDE5187EE0CE812F26177D00C026095AD7A8CEE9177EE1E3
S123E160A8CEE6A2BDE5187EE0CEBDE20720BAD7A8CEE54EDFB0DEB018CE008EE600C1FF80
S123E1802609CEE684BDE5187EE0CE3CCB033ADFB0385F5CA60118A10026DB081808D1A866
S123E1A02DF1DEB00909EE00AD007EE0CE81612D06817A2E02802039CE009CC6086F00080E
S123E1C05A2EFA39505958414243530002040607080901010100000001A600363CBDE3CABC
S123E1E0862DBDE3CAE607A60ECE00603A4D2703BDE4F0BDE4FF3832393CCEE1C4BDE1D984
S123E20008815326F8383936373CBDE1AD81302D2281392F0A81412D1A81462E168B09847C
S123E2200FCE0096C604680169005A2EF9AA01A70120037C00C0383332397F00C07F00A85C
S123E2407F00967F0097BDE306BDE2F1BDE2077D00C026087C00A8BDE2F820ED397F00A820
S123E2607F00967F0097BDE54481182704817F26037EE0CE7F00C0BDE2077D00C026057CA7
S123E28000A820E2397D00A827059697BDE290398C103F27109C9825129C9A220E37E600B1
S123E2A0C1FF332703BDE2C6BDE2BAA700A10027083CCEE69DBDE518383937C602F7103B0F
S123E2C0A700C603201837C616F7103BC6FFE700C617200A37C606F7103BA700C6072601AA
S123E2E05FF7103B333CCE0D060926FD387F103B393CDEAEA60038393CDEAE0820043CDED5
S123E300AE09DFAE3839BDE2F1BDE3162605BDE2F820F3810D39812C270681202702810934
S123E32039BDE3162702810D39BDE39E271881172605BDE39E27FB817F27088118270481E6
S123E3400126037EE0CE39368601B740003239368600B740003239CE00C418CEE371CC7ED7
S123E36003A1002705A7001AEF013A8C010026F139865006CF7EE371363C96A5810026052B
S123E380BDE449201681012605BDE488200DCED00081022703CED008BDE3F33832393C866D
S123E3A055B7103A86AAB7103A96A52605BDE459201681012605BDE494200DCED00081020C
S123E3C02703CED008BDE41E383936373CD6A52605BDE4662016C1012605BDE4AE200DCE76
S123E3E0D000C1022703CED008BDE4293833327C00A9398622A7028638A7028640A7028644
S123E40010A7028600B7D0048600B7D0058613A7008607A70086BBA7018605A70239A601AB
S123E42084012704A603847F397D00A427108D0E810D2604860A2006810A260C860DE601AB
S123E440C40427FA847FA703398630B7102B8600B7102C860CB7102D39B6102E8420270545
S123E460B6102F847F397D00A427108D0E810D2604860A2006810A260E860DF6102EC5803B
S123E48027F9847FB7102F39CE98008603A7008616A70039CE9800A6003684303227068639
S123E4A00197C2200484012704A601847F398D187D00A42712810D2606860A8D0B200881BD
S123E4C00A2604860D8D0139CE9800E600C50227F7847FA70139FFFFFFFFFFFFFFFF444415
S123E4E04444840F8B3081392F028B07BDE3CA3936A600368DE8328DE9320839BDE4F0BD32
S123E500E4F08620BDE3CA39860DBDE3CA8600BDE3CA860D7F00A939BDE50836A6008104EE
S123E5202714BDE3CA08BDE39E27F1811726EDBDE39E27FB20E6323936BDE50296A98114AA
S123E5402FF73239BDE39E4D27FABDE3CA3905415353454DEB2405425245414BE6EE0442C6
S123E560554C4BE7A90742554C4B414C4CE7AD0443414C4CF9FD0444554D50E7B6054545FD
S123E5804D4F44E84B0446494C4CE89B02474FFA560448454C50F60404484F5354FBD10495
S123E5A04C4F4144FC6F064D454D4F5259E903044D4F5645E9D7064F4646534554FD8307B2
S123E5C050524F43454544FA44085245474953544552FDC40653544F504154FB2C05545216
S123E5E0414345FAE706564552494659FC67013FF6040558424F4F54FE34017EFEAC0341C5
S123E600534DEB24024246E89B04434F5059E9D7054552415345E7A9024D44E7B6024D4D6A
S123E620E903025244FDC402524DFDC40452454144E9D702544DFBD10454455354FEADFFF2
S123E64042554646414C4F20332E34202865787429202D20426974205573657220466173BB
S123E6607420467269656E646C792041696420746F204C6F676963616C204F70657261742E
S123E680696F6E04576861743F04546F6F204C6F6E670446756C6C044F702D2004726F6D7A
S123E6A02D04436F6D6D616E643F0442616420617267756D656E74044E6F20686F737420DA
S123E6C0706F727404646F6E650463686B73756D206572726F72046572726F722061646477
S123E6E072200472637672206572726F7204BDE3062604BDE78539812D2631BDE2F8BDE208
S123E700F1BDE3212606BDE1B87EE6EEBDE23ABDE3212707CEE6ABBDE51839BDE7945D2B95
S123E72008CE009C3A6F006F017EE6EEBDE23ABDE3212707CEE6ABBDE51839BDE7945D2C1D
S123E740ADDE96A60036863FBDE290E60032BDE290C13F270CDFB0CE00B0BDE4FCBDE78577
S123E760397F00967F00973CBDE794385D2A0ACEE693BDE518BDE7853918CE009C183ACDF0
S123E780EF007EE6EEBDE508CE009CC604BDE4FC5A2EFA395FCE009C3AEE009C962601397B
S123E7A05C5CC1062FEFC6FF39DE982003CE103F86FFBDE2D439DEAADFB0C6803ADFB2BDEE
S123E7C0E3062735BDE23A7D00A82726BDE3212621DE96DFB0C6803ADFB2BDE306271ABDE5
S123E7E0E23A7D00A8270BBDE3062606DE96DFB22007CEE6ABBDE51839DCB0DDAAC4F0DDAE
S123E800B0BDE508CE00B0BDE4FCDEB05FBDE4FF5CC1102DF85FDEB03AA600812025048188
S123E8207A23028620BDE3CA5CC1102DE9BDE329DCB0C30010DDB01A93B2220E1A83000001
S123E84026BFDCB21A83FFF025B739BDE3062734BDE23A7D00A8273CBDE3212637DC96DDD1
S123E860B0C307FFDDB2BDE3062711BDE23A7D00A82721BDE306261CDE96DFB2DEB0DF9876
S123E880DEB2DF9ABDE508CE0098BDE4FCCE009ABDE4FC39CEE6ABBDE51839BDE306BDE2E9
S123E8A03A7D00A8274FBDE316264ADE96DFB0BDE306BDE23A7D00A8273BBDE3212636DE55
S123E8C096DFB286FF97C1BDE3062711BDE23A7D00A82721BDE306261C969797C1BDE329D6
S123E8E0DEB096C1BDE290A10026119CB2270508DFB020E939CEE6ABBDE51839CE00B0BD48
S123E900E4FC39BDE3062718BDE23ABDE3062707CEE6ABBDE518397D00A82704DE96DFAAA9
S123E920BDE508CE00AABDE4FCDEAABDE4FF7F00967F0097BDE25DBDE1ADDEAA81202731F9
S123E940810A273E812B2743815E2748812D274481082740812F2745813D2741814F2743DA
S123E960810D276F812E276ECEE6A2BDE5187EE920BDE28508DFAA8FC40F27037EE9297E45
S123E980E920BDE28508DFAA7EE923BDE28508DFAA7EE920BDE28509DFAA7EE920BDE2858E
S123E9A07EE920DC9693AA81002606C1802313200881FF2604C1812409CEE68ABDE5187E42
S123E9C0E920830001D7C3BDE502CE00C3BDE4FF7EE920BDE28539BDE23A7D00A8272BBD46
S123E9E0E3162626DE96DFB0BDE23A7D00A8271ABDE3212615DE96DFB2BDE23ABDE30626E6
S123EA00097D00A8270BDE96200ACEE6ABBDE51839DEB008DFB4DEB49CB023289CB22224BC
S123EA20DCB293B0D3B4DDB4DEB2BDE329A6003CDEB4BDE290A100262809DFB4389CB027B7
S123EA401F0920E6DEB0BDE329A6003CDEB4BDE290A100260C08DFB4389CB227030820E65E
S123EA603938CE00B4BDE4FC39EA7BEA8EEAA1EAB0EABDEAD0EAE8EB03EB10496D6D6564BF
S123EA80206D6F646520696C6C6567616C044572726F7220696E204D6E65207461626C6546
S123EAA004496C6C6567616C20626974206F700442616420617267756D656E74044D6E6584
S123EAC06D6F6E6963206E6F7420666F756E6404556E6B6E6F776E2061646472657373690C
S123EAE06E67206D6F646504496E64657865642061646472657373696E6720617373756D26
S123EB0065640453796E746178206572726F72044272616E6368206F7574206F66207261A1
S123EB206E676504CE0000DFBEBDE3062713BDE23ABDE3062707CEEAB0BDE51839DE96DFED
S123EB40BEDEBEDFB0BDE508CE00B0BDE4FCBDF376BDE538863EBDE4ECBDEC0597BC815ED2
S123EB602715812B2711812D270D812F2709813D27058100260439BDE508BDE502BDE502EF
S123EB80BDE502BDE502BDE502BDEC4EC1052F08CEEABDBDE518202FC100272EBDEC959629
S123EBA0B581FF2608CEEABDBDE518201ABDECCD81002607CE0000DFB6200F4A16CEEA694E
S123EBC03A3AEE00BDE5187F00BC96BC815E2704812D2607DEBE09DFBE2027810A270881DF
S123EBE02B2704810D261BDEB62606DEB0DFBE2011810A2704812B2605DEBE08DFB6DEB676
S123EC00DFBE7EEB415F860DCE006B3AA7005CC1232DF55FBDE544817F27318118272D8130
S123EC20012729812E2725810327218104271D810826055A2EDE20CDCE006B3ABDE1ADA783
S123EC4000C1232C015CBDEC7A26C9394F3986209791CE006BDFAEBDE3065FBDE2F1BDE2A8
S123EC60F8BDE3162713BDEC7A270EBDE1ADCE008E3AA7005CC1052FE239810A2716810D06
S123EC802712815E270E812F270A812B2706812D2702813D39CEEFF718CE008E2003C60684
S123ECA03AA6008104260586FF97B53918A10026EDA60118A10126E6A60218A10226DFA66F
S123ECC00318A10326D8EC0497B4D7B539860497C17F00C2DEAE8C008E271BEC0008812CC7
S123ECE026F4C1592606860297C1200AC1582606860197C12000BDE30681232607BDE2F854
S123ED00860097C1D6B5C10226037EED6BC10126037EED70C10526037EED77C10826037EBD
S123ED20EDA6C10726037EEDB0C10326037EEDB9C10426037EEDC7C11526037EEDF9C110CB
S123ED4026037EEE1AC10926037EEE23C11226037EEE3BC11126037EEE44C11326037EEEC7
S123ED6063C11426037EEE638602398618BDEFEC96B4BDEFEC4F39BDEFCE8104260139DCC3
S123ED8096DEB00808DFB893B8DDB81A83007F23091A83FF80240386093996B4BDEFEC96F9
S123EDA0B9BDEFEC4F3996C181002604860397C196C181002603860139860097C397B28623
S123EDC01897B3BDEEFF3996C1810226098618BDEFEC860197C196C181012604BDEF9F3945
S123EDE096B48B10BDEFECBDEFCE8104270ADC96BDEFEC17BDEFEC4F3996C1810026048699
S123EE000397C196C1810226037C00C2861A97C397B286CD97B3BDEEFF3996C1810026038E
S123EE2086013996C181002604860397C1860097C397B286CD97B3BDEEFF3996C181002684
S123EE400386013996C1810226037C00C281002604860397C1861897C397B3861A97B2BD36
S123EE60EEFF39BDEED98100260386033996C1810226098618BDEFEC860197C196B4BDEF64
S123EE80ECBDEFCE81042601399697BDEFEC96C181012606BDE2F8BDE2F8BDEFCE81042606
S123EEA001399697BDEFEC96B5811426024F39BDEFCE8104260139DEB008DFB8DC9693B876
S123EEC01A83007F230D1A83FF8024074FBDEFEC86093917BDEFEC4F3996C1D6B58101262B
S123EEE001398102260139C114260796B4800897B439C113260796B4800C97B4394F399620
S123EF00C1810327138100272C810227418101274C8104275786063996C3BDEFE496B4BD02
S123EF20EFECBDEFCE8104260139DC96BDEFEC17BDEFEC4F3996C3BDEFE496B4BDEFECBDCA
S123EF40EFCE81042601399697BDEFEC4F3996B3BDEFE496B48B2097B4BDEF9F3996B2BD1C
S123EF60EFE496B48B2097B4BDEF9F39BDEFCE810426013996C3BDEFE496A881022E0E961B
S123EF80B48B10BDEFEC9697BDEFEC4F3996B48B30BDEFECDC96BDEFEC17BDEFEC4F3996C5
S123EFA0B4BDEFECBDEFCE8104260139812C2703860839BDE2F8BDE2F18159270A815827D2
S123EFC006FEEAE8BDE5189697BDEFEC4F39BDE23ABDEC7A2705BDE31626067D00A82701F9
S123EFE03986043981002703BDEFEC39DEB0BDE290BDE4FFDFB039414241201B0141425895
S123F000203A01414259203A0241444341890341444342C903414444418B0341444442CB80
S123F0200341444444C308414E44418403414E4442C40341534C20680441534C4148014163
S123F040534C42580141534C44050141535220670441535241470141535242570142434320
S123F06020240542434C521D14424353202505424551202705424745202C05424754202E5F
S123F0800542484920220542485320240542495441850342495442C503424C45202F05422D
S123F0A04C4F202505424C53202305424C54202D05424D49202B05424E4520260542504CE4
S123F0C0202A054252412020054252434C1F1342524E202105425253451E13425345541C9F
S123F0E014425352208D05425643202805425653202905434241201101434C43200C0143C4
S123F1004C49200E01434C52206F04434C52414F01434C52425F01434C56200A01434D50CE
S123F120418103434D5042C103434F4D206304434F4D414301434F4D425301435044208367
S123F14015435058208C09435059208C11444141201901444543206A04444543414A014457
S123F1604543425A01444553203401444558200901444559200902454F52418803454F5285
S123F18042C803464449560301494449560201494E43206C04494E43414C01494E43425CB8
S123F1A001494E53203101494E58200801494E592008024A4D50206E044A5352208D074C74
S123F1C044414186034C444142C6034C444420CC084C4453208E084C445820CE094C4459D7
S123F1E020CE114C534C2068044C534C4148014C534C4258014C534C4405014C53522064F0
S123F200044C53524144014C53524254014C53524404014D554C203D014E45472060044EB5
S123F22045474140014E45474250014E4F502001014F5241418A034F524142CA03505348B4
S123F240413601505348423701505348583C01505348593C0250554C41320150554C423300
S123F2600150554C58380150554C593802524F4C206904524F4C414901524F4C42590152B6
S123F2804F52206604524F52414601524F52425601525449203B01525453203901534241C4
S123F2A020100153424341820353424342C203534543200D01534549200F01534556200B69
S123F2C00153544141870753544142C70753544420CD0753544F50CF01535453208F075382
S123F2E0545820CF1053545920CF1253554241800353554242C00353554244830853574915
S123F300203F01544142201601544150200601544241201701545041200701544553540013
S123F32001545354206D04545354414D01545354425D015453582030015453592030025421
S123F3405853203501545953203502574149203E01584744588F01584744598F0242525392
S123F3604512164252434C131642534554141742434C52151704DEB0A600C6008118270A60
S123F380811A270581CD26045C5C5C08DFB6D7C3A60097B408DFB6815F230F818D270B817E
S123F3A08F270781CF27037EF441D6C3C1022504BDF5FB39D6B45FBDF52A5D2604BDF5FBFB
S123F3C03996B4818D2604C605200A818F270481CF2605C601BDF52AD6B5C1012618D6C3FC
S123F3E0C100270E96B4C602BDF52A5D2604BDF5FB39BDF54D39D6B5C10526107D00C32792
S123F40004BDF5FB39BDF54DBDF58339D6B5C1172704C11626117D00C32704BDF5FB39BDE7
S123F420F54DBDF5DB2006BDF54DBDF567BDE502BDF5DBD6B5C1132704C1162603BDF583CB
S123F44039817F222AD6C3C1022504BDF5FB39846F5FBDF52A5D2604BDF5FB39BDF54D9688
S123F460B484F081602604BDF56739BDF5E8398187270481C72604BDF5FB3984CF5FBDF541
S123F4802A5D2604BDF5FB3996B484CF818D2604C6072016818F2604C607200E81CF26044A
S123F4A0C61020068183260CC608BDF52A5D2604BDF5FB39D6B5C1032708C1072704C108C5
S123F4C0263196B484CF8183260FD6C3C1022509C615BDF52AC608D7B5D6C3C1012704C119
S123F4E003260C96B484B081A02704BDF5FB39BDF5A539D6C3C1012704C102261396B48443
S123F500CFD6B5C1092604C6112002C612BDF52AD6C3C102250C96B484B081A02704BDF5E3
S123F520FB39C608D7B5BDF5A539CEEFF7A104260F5D2704E1052608E605D7B5DFBA5C39DA
S123F54037C6063AE600C1043326E25F39DEBAA600BDE4ECA601BDE4ECA602BDE4ECA6030F
S123F560BDE4ECBDE50239BDF5DB862CBDE4ECD6C3C1012704C1032604865920028658BD41
S123F580E4EC39DEB6E60008DFB65D2B033A2004095C26FCDFB8BDE5028624BDE4ECCE0097
S123F5A0B8BDE4FC39BDF54D96B484B0818026178623BDE4ECBDF5DBD6B5C108270139DEA8
S123F5C0B6BDE4F0DFB63981902604BDF5DB3981A02604BDF56739BDF5E8398624BDE4EC6A
S123F5E0DEB6BDE4F0DFB6398624BDE4ECDEB6BDE4FCDFB639494C4C4F50043CCEF5F5BDA9
S123F600E51B3839CEF60BBDE5183941534D205B3C616464723E5D20204C696E6520617329
S123F6206D2F64697361736D0D20205B2F2C3D5D202053616D6520616464722C20202020DF
S123F6402020205B5E2C2D5D20205072657620616464722C202020202020205B2B2C4354EA
S123F6604C4A5D204E65787420616464720D20205B43525D20204E657874206F70636F646B
S123F680652C20202020202020202020202020202020202020202020202020202020202015
S123F6A05B43544C412C2E5D2020517569740D4246203C61646472313E203C616464723209
S123F6C03E205B3C646174613E5D2020426C6F636B2066696C6C206D656D6F72790D4252B0
S123F6E0205B2D5D5B3C616464723E5D2053657420757020626B7074207461626C650D429B
S123F700554C4B2020457261736520454550524F4D2C2020202020202020202020202020F5
S123F72020202042554C4B414C4C2020457261736520454550524F4D20616E6420434F4EF3
S123F7404649470D43414C4C205B3C616464723E5D2043616C6C20737562726F7574696E12
S123F760650D474F205B3C616464723E5D204578656375746520636F646520617420616408
S123F78064722C202020202020202050524F434545442020436F6E74696E7565206578657A
S123F7A0637574696F6E0D45454D4F44205B3C616464723E205B3C616464723E5D5D204DF5
S123F7C06F6469667920454550524F4D2072616E67650D4C4F41442C205645524946592087
S123F7E05B545D203C686F73742064776E6C6420636F6D6D616E643E20204C6F6164206F1A
S123F800722076657269667920532D7265636F7264730D4D44205B3C61646472313E205B51
S123F8203C61646472323E5D5D20204D656D6F72792064756D700D4D4D205B3C616464723B
S123F8403E5D206F72205B3C616464723E5D2F20204D656D6F7279204D6F646966790D207E
S123F860205B2F2C3D5D202053616D6520616464722C20205B5E2C2D2C43544C485D2050F1
S123F88072657620616464722C20205B2B2C43544C4A2C53504143455D204E6578742061DC
S123F8A06464720D20203C616464723E4F20436F6D70757465206F66667365742C20202029
S123F8C0202020202020202020202020202020205B43525D2020517569740D4D4F56452090
S123F8E03C73313E203C73323E205B3C643E5D2020426C6F636B206D6F76650D4F464653B4
S123F9004554205B2D5D3C6172673E20204F666673657420666F7220646F776E6C6F61640B
S123F9200D524D205B502C592C582C412C422C432C535D20205265676973746572206D6F9C
S123F940646966790D53544F504154203C616464723E2020547261636520756E74696C203F
S123F960616464720D54205B3C6E3E5D20205472616365206E20696E737472756374696F96
S123F9806E730D544D20205472616E73706172656E74206D6F6465202843544C41203D2054
S123F9A0657869742C2043544C42203D2073656E642062726B290D5B43544C575D202057D3
S123F9C06169742C202020202020202020205B43544C582C44454C5D2041626F727420202D
S123F9E0202020202020205B43525D20526570656174206C61737420636D640D04BDE30676
S123FA002713BDE23ABDE3062707CEE6ABBDE51839DE96DF60DE6909CCFA29ED0009DF6979
S123FA20BDFA9A7F00C17EFB89360797680F32DD66DF6418DF629F699EB2BDFAC7BDE50853
S123FA40BDE1F939BDFB69BDE3297F00C17C00C1BDFA9A7EFB89BDE3062713BDE23ABDE3BF
S123FA60062707CEE6ABBDE51839DE96DF607F00C17C00C1BDFA9A7EFB89309EB2BDFBA899
S123FA80BDFAC7DE6009DF607D00C12606DE690808DF69BDE508BDE1F9395FCE009C18CE2C
S123FAA000B63A183AEE00270AA60018A700863FBDE290CB02C1062FE2DEF5DFB4867E97E2
S123FAC0F4CEFA7ADFF5395FCE009C18CE00B63A183AEE00270618A600BDE290CB02C10652
S123FAE02FE6DEB4DFF5397F00C37C00C37F00A9BDE3062713BDE23ABDE3062707CEE6ABB9
S123FB00BDE51839969797C3D6C337DE60DFB0BDF37633D7C3BDFB69BDE329BDE538BDE175
S123FB20F97A00C32705BDE50820DD39BDE3062718BDE23ABDE3062707CEE6ABBDE518399B
S123FB407D00A82704DE96DFAADC601A93AA250ADCAAC3000A1A93602208BDFB69BDE3291E
S123FB6020E7BDE508BDE1F939867E97D3CEFBA5DFF2966884BF9768C657FE100E3AFF1091
S123FB801EB6102084FEB71020BF00B2BE0069FE00603CFE00623CFE00643CFC00663637B9
S123FBA0B60068363B309EB2A6009768EC019767D766EC03DD64EC05DD62EC07DD60C60807
S123FBC03ADF69B610208A03B710208608B7100B3996A62607CEE6B8BDE518397F00A4BD04
S123FBE0E347BDFC41BDE39E4D27108101271781022605BDFC0D2003BDFC59BDFC4D4D2738
S123FC00E4BDE3CA20DF7C00A4BDE34F3996A78103270DCE102D1C00018D1D1D0001200D39
S123FC20CED0088660A7028D0F8670A702860DBDFC59860ABDFC593918CE6F9B180926FC9D
S123FC4039D6A537D6A7D7A5BDE3782016D6A537D6A7D7A5BDE39E200AD6A537D6A7D7A5B0
S123FC60BDE3CA33D7A5397F00C17C00C120037F00C17F00C2BDE30626037EFBD1BDE1ADA9
S123FC8081542616BDE2F8BDE2F1BDE2FE810D26097F00A496A597A7201B7F00A4BDE347ED
S123FCA0BDFC41BDE2F1BDE2F836BDFC59BDE3CA32810D26EE96A791A52703BDE329BDFC7A
S123FCC04D4D27F1815326EDBDFC4D4D27FA8139274E813126DF7F00C3BDFD66D697C0029C
S123FCE0BDFD66BDFD6637DC96D3AC8F3309BDFD66085A271B7D00C226BB7D00C1260596EA
S123FD0097BDE290A10027E6860297C2DFB420DE7D00C226A096C34C279B860397C22095F6
S123FD20BDFD66D697BDFD665A26FAC664BDE2E55A26FABDE39ECC7E0DDD6B7C00A4BDE3D3
S123FD404FCEE6C596C281022608CE00B4BDE4FC201381012605CEE6E3200781032603CE96
S123FD60E6CABDE51839373CBDFC4D4D27FABDE207BDFC4D4D27FABDE20796979BC397C350
S123FD803833397F00C3BDE3062728812D26097C00C3BDE2F8BDE306BDE23A7D00A8271DE9
S123FDA0BDE3062618DC967D00C32705CC00009396DDACBDE508CE00ACBDE4FC39CEE6ABA6
S123FDC0BDE51839CEE1C4BDE306BDE1AD810D271CA100270EE60008C15326F5CEE6ABBDE8
S123FDE0E518393CBDE2F8BDE3063826EFBDE1F9BDE508BDE1D97F00967F0097BDE25DBD67
S123FE00E3212707CEE6ABBDE51839363C7D00A82714E607A60ECE00603A4D27059696A733
S123FE2000089697A7003832E600C153270508810D26BD39BDE306260BCEC0FFDFB818CEBF
S123FE40C0002036BDE23A7D00A8272718DE96BDE306260C18DFB8DCB8C300FFDDB8201A04
S123FE60BDE23A7D00A8270BDE96DFB8BDE30626022007CEE6ABBDE51839C6FFBDFE9218D2
S123FE80A600A72F1F2E80FC189CB82704180820EE39CE10008602A708A7096F2D8622A76B
S123FEA02B860CA72DE72F1F2E80FC393986FFB710007F00A4BDE347BDFC41867FBDFC59F5
S123FEC0860DBDFC597C00A4CE0070DFAE18CEFEEB18A60081042707A70008180820F27FEE
S11FFEE000C1BDFC9A8E005F7EC0B363617420657662746573742E6F75740D0424
S123FF7C7EE0CE7EE1B87EE1F97EE2077EE23A7EE25D7EE2857EE2F17EE2F87EE2FE7EE3BB
S107FF9C067EE329CD
S123FFA07EE1AD7EE3167EE3217EE3787EE39E7EE3CA7EE4DE7EE4E27EE4EC7EE4F07EE4AF
S116FFC0FF7EE4FC7EE5087EE5187EE51B7EE5447EE3570A
S123FFD600C400C700CA00CD00D000D300D600D900DC00DF00E200E500E800EB00EE00F15F
S10DFFF600F400F700FA00FDE0003B
S9030000FC
